:100000000C9446000C9465000C9465000C946500FB
:100010000C9465000C9465000C9465000C946500CC
:100020000C9465000C946E000C9465000C946500B3
:100030000C9465000C9465000C9465000C946500AC
:100040000C9465000C9465000C9465000C9465009C
:100050000C9465000C9465000C9465000C9465008C
:100060000C9465000C9465000C9465000C9465007C
:100070000C9465000C9465000C9465000C9465006C
:100080000C9465000C94C7030C94650011241FBEEA
:10009000CFEFD0E1DEBFCDBF11E0A0E0B1E0E2E400
:1000A000FCE000E00BBF02C007900D92A030B1074A
:1000B000D9F711E0A0E0B1E001C01D92A33FB10764
:1000C000E1F70E948A000C941F060C9400008BE05C
:1000D00085BD89EF83BD80E887BF08951F920F9289
:1000E0000FB60F9211248F939F93809100019091EE
:1000F0000101019690930101809300019F918F91DE
:100100000F900FBE0F901F90189585B394E089272C
:1001100085BB0895EF92FF920F931F938FEF84BBDF
:10012000F89484E08093F20180E090E060E070E079
:100130000E94A4030E9492030E9467000E947F0114
:1001400080E090E060E070E00E94F50085E890E0DB
:1001500060E070E040E050E021E030E004EF11E0CA
:10016000E2E3EE2EF12C0E94C70186E091E060E010
:1001700070E040E050E021E030E00AE010E0EE24E2
:10018000FF240E94C70178940E94A702FDCFFC01C2
:1001900083899489029741F5828190E09C012078BF
:1001A000307087FF04C020383105F1F417C0238177
:1001B0008281628190E08F709070982F882730E064
:1001C00070E060717070F4E075956795FA95E1F7ED
:1001D000822B932B70E00E9494010895828190E01D
:1001E00060E070E00E946901089584B3836084BB7D
:1001F00085B38C7F85BB1ABA8FEF8BBB82E080936F
:100200000201089585B38C7F85BB0895DF93CF935A
:1002100000D0CDB7DEB7C99906C0A8988091020179
:100220008130C9F408C0C89913C0A998809102010F
:10023000813089F482E08A8384E0898381E0BE0191
:100240006F5F7F4F42E00E94C4051092020103C01D
:1002500081E0809302010F900F90CF91DF9108957C
:10026000DF93CF9300D0CDB7DEB7C89B06C0A89868
:10027000A99A81E0809302010BC084E0898382E027
:100280008A8381E0BE016F5F7F4F42E00E94C40518
:100290000F900F90CF91DF910895DF93CF9300D00F
:1002A000CDB7DEB7C99B06C0A998A89A81E0809314
:1002B00002010AC084E0898381E08A83BE016F5F06
:1002C0007F4F42E00E94C4050F900F90CF91DF91C5
:1002D000089581FF10C080FF07C080E090E060E0DB
:1002E00070E00E944D01089580E090E060E070E0D1
:1002F0000E943001089585B38C7F85BB089587B334
:10030000806C87BBC09A88E28FBD82E18EBD80E29F
:100310009EE497BD86BD8CED95E099BD88BD909318
:100320007900809378000895672B19F499BD88BDF2
:10033000089590937900809378000895089588B582
:1003400099B5895E934050F41AC088B599B5019764
:1003500099BD88BDC9010197F1F702C020E137E2DC
:1003600088B599B5885E934081F7089588B599B5A9
:10037000019699BD88BDC9010197F1F702C020E13E
:1003800037E288B599B58056994081F70895CF92A4
:10039000DF92EF92FF920F931F93CF93DF93EC01C5
:1003A0006901A0E0B0E09A2FFD0184E0EE0FFF1F8D
:1003B0008A95E1F7EA1BFB0BED5FFE4F85858823ED
:1003C00029F09F5F1196AC30B10569F7292F30E015
:1003D000F901A4E0EE0FFF1FAA95E1F7E21BF30B72
:1003E000ED5FFE4FD183C083738362835583448363
:1003F000D782C682E114F10411F4168608C082E3A4
:10040000E816F10411F481E001C082E08687F90169
:1004100054E0EE0FFF1F5A95E1F7E21BF30BED5F7F
:10042000FE4FA685B0E0A954BE4F8C91982F9E0D2B
:1004300094878F5F8C931187008781E08587F8947C
:100440008091000190910101800F911FF90144E01A
:10045000EE0FFF1F4A95E1F7E21BF30BED5FFE4F36
:10046000938782877894DF91CF911F910F91FF90AE
:10047000EF90DF90CF900895CF92DF92EF92FF92AE
:100480000F931F93CF93DF93EC01690120E030E0DD
:10049000A22FF901B4E0EE0FFF1FBA95E1F7E21BBE
:1004A000F30BED5FFE4F8585882331F0AF5F2F5F43
:1004B0003F4F2C30310561F72A2F30E0F901A4E0DD
:1004C000EE0FFF1FAA95E1F7E21BF30BED5FFE4F66
:1004D000D183C0837383628355834483D782C6826A
:1004E000E114F10411F4168608C082E3E816F10461
:1004F00011F481E001C082E08687D90194E0AA0F5F
:10050000BB1F9A95E1F7A21BB30BAD5FBE4FED0188
:10051000EE85F0E0E954FE4F8081982F9E0D9C8778
:100520008F5F80831987088781E08D878091000124
:1005300090910101800F911F9B878A87DF91CF9156
:100540001F910F91FF90EF90DF90CF900895CF9380
:10055000DF93F894609100017091010178941092FA
:10056000BA018091BD018F5F8093BD018091BD0173
:10057000883C49F48091BC0186958093BB01109220
:10058000BC011092BD014FEF5FEF20E030E0F901B8
:10059000A4E0EE0FFF1FAA95E1F7E21BF30BED5F5E
:1005A000FE4F8585882379F08091BA018F5F809313
:1005B000BA01828593856817790728F084858517A5
:1005C00010F45485422F2F5F3F4F2C303105F9F640
:1005D0004F3F79F18091BC018F5F8093BC01842FE4
:1005E000992787FD9095EC0124E0CC0FDD1F2A951B
:1005F000E1F7C81BD90BCD5FDE4FE881F9818A8115
:100600009B816C817D8109958E819F81892B49F425
:100610001D86EE85F0E0E954FE4F80818150808395
:1006200008C02A853B8588859985820F931F9B8703
:100630008A8781E0DF91CF910895AC0120E030E01E
:10064000F90184E0EE0FFF1F8A95E1F7E21BF30B3F
:10065000ED5FFE4F8081918184179507C1F48585F8
:100660008823A9F0F8948091000190910101860FF0
:10067000971FF901B4E0EE0FFF1FBA95E1F7E21BF7
:10068000F30BED5FFE4F93878287789408952F5F79
:100690003F4F2C303105A1F60895AC0120E030E049
:1006A000F90194E0EE0FFF1F9A95E1F7E21BF30BBF
:1006B000ED5FFE4F808191818417950761F48585F8
:1006C000882349F08091000190910101860F971FC6
:1006D0009387828708952F5F3F4F2C30310501F7B4
:1006E0000895AC0120E030E0F90164E0EE0FFF1F57
:1006F0006A95E1F7E21BF30BED5FFE4F808191817C
:100700008417950749F41586E685F0E0E954FE4F15
:1007100080818150808308952F5F3F4F2C303105B9
:1007200019F7089580E090E0FC0174E0EE0FFF1FE0
:100730007A95E1F7E81BF90BED5FFE4F1586019600
:100740008C30910589F708958091F201880F8160BE
:100750008093720080E480937000E1E7F0E0808194
:100760008C7F80832FEF2093730085EC809374003F
:1007700081E090E09093C1018093C0011092BF018D
:100780002093EC011092D6011092D50108951F928A
:100790000F920FB60F920BB60F921124EF92FF92A9
:1007A0000F931F932F933F934F935F936F937F9379
:1007B0008F939F93AF93BF93EF93FF938091C0016B
:1007C0009091C101817C09F4BFC08091710090E0DB
:1007D000887F90708036910509F49CC08836910519
:1007E00009F480C08037910509F494C088379105D9
:1007F00009F478C08038910581F08838910509F4B2
:1008000099C08039910549F08839910509F492C061
:10081000803A910509F096C093C08091C0019091F3
:10082000C1018034910581F4809173008093C301EC
:100830008FEF8093EC0180E890E09093C10180936A
:10084000C0011092BF017CC08091C0019091C10194
:100850008038910509F074C09091BF018091C30167
:100860009817A0F48091BF01E82FF0E090917300F9
:10087000EE53FE4F92838F5F8093BF019091EC0106
:100880008091730089278093EC015AC08091BF0149
:10089000803111F5809173008093D4019091EC0127
:1008A0008091D401981719F081E090E002C082E0B5
:1008B00090E09093D6018093D50187EC90E062ECB4
:1008C00071E040E050E020E030E000E010E0EE2495
:1008D000FF240E943C022EC08091BF018F5F809355
:1008E000BF012EC08091F0018F5F8093F001809155
:1008F000ED018A3078F48BE895E060E070E040E04C
:1009000050E020E030E002E310E0A2E3EA2EF12C18
:100910000E943C02809173008093C2011092D60124
:100920001092D5011092BF0185EC8093740080E491
:1009300090E078C081E090E09093C1018093C00185
:1009400085ECD0C085E4CEC08091710090E0887FB6
:10095000907088309105A9F08031910591F088312F
:100960009105C9F08032910509F48EC08832910555
:10097000C9F08033910509F45AC0C89709F0ABC09B
:100980005CC08091D7018093730085E880937400E8
:1009900088E090E047C01092BE018091D80180931A
:1009A00073003BC08091BE018131D9F485E9809309
:1009B000740080E290E09093C1018093C001109296
:1009C000ED018091EE019091EF0101969093EF017E
:1009D0008093EE0184EA93E060E070E00E944D03B2
:1009E00083C09091BE018091D801981750F08091FA
:1009F000E901809373008091BE018F5F8093BE01F7
:100A00000CC09091BE01E92FF0E0E952FE4F8281C7
:100A1000809373009F5F9093BE0185E8809374007C
:100A200080E190E09093C1018093C0015DC080910E
:100A3000F0018F5F8093F0012CC08091F0018F5FF7
:100A40008093F00184EA93E060E070E00E944D033F
:100A50008091ED018A3080F48BE895E060E070E0F1
:100A600040E050E020E030E002E310E0F2E3EF2E5F
:100A7000F12C0E943C0206C088E290E09093C101F4
:100A80008093C00185E82EC08091F1018F5F809333
:100A9000F10184EA93E060E070E00E944D038091F0
:100AA000ED018A3080F48BE895E060E070E040E092
:100AB00050E020E030E002E310E0E2E3EE2EF12C23
:100AC0000E943C0206C088E290E09093C1018093AE
:100AD000C00185E907C084E090E09093C101809354
:100AE000C00185E080937400FF91EF91BF91AF91B9
:100AF0009F918F917F916F915F914F913F912F9136
:100B00001F910F91FF90EF900F900BBE0F900FBEB3
:100B10000F901F901895EF92FF920F931F93809163
:100B2000C0019091C101019759F08BE895E060E018
:100B300070E040E050E020E030E005E010E01AC056
:100B40001092BE0185EA8093740082E090E0909359
:100B5000C1018093C0018091ED018F5F8093ED0111
:100B600084EA93E060E070E040E050E020E030E0B4
:100B700000E117E2B2E3EB2EF12C0E94C7011F91B6
:100B80000F91FF90EF900895EF92FF920F931F93B4
:100B9000582F8091ED01882309F448C08091ED0120
:100BA0008A3009F443C081E03CC08FEF8093E901B3
:100BB000DB0120E030E00DC08C91F901E952FE4FDD
:100BC00082838091E9019D9189278093E9012F5FBC
:100BD0003F4F241788F381E08093ED01852F90E04B
:100BE000880F991F8093D7014093D8011092BE01BE
:100BF00085EA8093740082E090E09093C101809335
:100C0000C00184EA93E060E070E040E050E020E062
:100C100030E005E010E0E2E3EE2EF12C0E94C70187
:100C200080E01F910F91FF90EF9008958091C00197
:100C30009091C101019709F4B8CF82E0F2CFF89406
:020C4000FFCFE4
:00000001FF
